:020000040000FA
:0400000028280000AC
:020008000528C9
:06000A00F0000308A20053
:100010000A08A3000408A4008B1C1E280708F2008D
:10002000720E0F39740784000008F50072080F394A
:10003000730784007508800086088B1083012408EC
:10004000840023088A0022088300F00E700E090045
:100050002530F3003530F400831603138117831223
:10006000031385018601870183160313013086007F
:10007000FF3087008501831203138601003085005D
:100080007E30B5000C30B600B630B7009E30B800F8
:10009000CC30B900DA30BA00F830BB000E30BC000A
:1000A000FE30BD00CE30BE000030BF008030C0004A
:1000B000FA30C100F030C200BC30C3001030C400C0
:1000C000831603130113831203130B168B172530AA
:1000D00084001030A0000030A1007528000000004E
:1000E000000000000000000000006430F200F20B8D
:1000F000772886012108850000088600A10A840A65
:06010000A00B6E28672829
:04010600003400348D
:02400E007A3FF7
:00000001FF
